:020000020000FC
:0400000007C0ACC0C9
:10000C004DC0B6C00FED0DBF0CEF07BB03E008BB36
:10001C0003E701BB0CE002BB02E005BF02E0B09BB2
:10002C0002E0B19B01E003BF0AE9B09B0EECB19B6F
:10003C0000E4B09903C0B19901C007E8002E02BEDC
:10004C0000E008BF09BF08E90AB903E3B09B09E166
:10005C00B19B0CE0B09903C0B19901C008E009B99B
:10006C002227E0E6F0E0C0E6D0E08827ACE9B0E07B
:10007C000CE9302E00E0402E992700E40BBF789459
:10008C0024FD01D0FDCF5D9BFECF5D91A83D08F016
:10009C00ACE95CB99A9509F42F7E08951FB602BE9F
:1000AC0025FD01C032C026FF1CC010FF949A000031
:1000BC000000000000000000000000000000000034
:1000CC000000000094987A9519F0169510681CC0E1
:1000DC002F7B8A95C9F42F7D02BE00E008BF09BFB3
:1000EC0013C01991CC3908F0C0E6206479E0949AD9
:1000FC0000000000000000000000000000000000F4
:10010C00000000000000949821C020FF1FC022FFB7
:10011C0019C021FD4F772D7F3A9519F0469540680F
:10012C0015C0AF93A32D4D93A83D08F0ACE9939562
:10013C003A2EAF9102BE00E008BF09BF20612B7FB1
:10014C002E7F04C024602D7F38E04FEF1FBE189522
:10015C001FB625FD0BC020FF02C0226007C0216026
:10016C00602D625E62BF02E008BF09BF1FBE18951A
:10017C002FB66CB16193EC3908F0E0E68395206200
:10018C002E7F2B7F02BE02E008BF09BF2FBE189541
:00000001FF
